:020000040800F2
:10300000A04A002001310008E56A0008A567000811
:10301000E16A0008413300083D7F0008000000001D
:10302000000000000000000000000000E16C00084B
:10303000B33B000800000000216B0008996D0008F8
:103040001B3100081B3100081B3100081B31000830
:103050001B3100081B3100081B3100081B31000820
:103060001B3100081B3100081B310008753B0008AC
:103070001B3100081B3100081B3100081B31000800
:103080001B3100081B3100081B3100081B310008F0
:10309000B97A00081B3100081B3100081B310008F9
:1030A0001B3100081B3100081B3100081B310008D0
:1030B0001B3100081B3100081B3100081B310008C0
:1030C0001B3100081B3100081B3100081B310008B0
:1030D0001B310008A97900081B310008CD790008D0
:1030E0001B3100081B3100081B310008DFF80CD031
:1030F00000F05CF800480047ED810008A04A00207D
:103100000648804706480047FEE7FEE7FEE7FEE781
:10311000FEE7FEE7FEE7FEE7FEE7FEE7516E00088A
:10312000ED300008202A04DB203A21FA02F00021C9
:10313000704721FA02F3D040C2F1200291400843C7
:103140001946704740EA01039B0703D009E008C90C
:10315000121F08C0042AFAD203E011F8013B00F85C
:10316000013B521EF9D27047D2B201E000F8012BA8
:10317000491EFBD270470022F6E710B513460A46F7
:1031800004461946FFF7F0FF204610BD30B505464E
:103190000020034600E05B1C934205D2EC5CC85C57
:1031A000201A01D1002CF6D130BD0000064C074D8D
:1031B00006E0E06840F0010394E807009847103407
:1031C000AC42F6D3FFF796FFB08D0008D08D000813
:1031D00070B5044600252068806800F00100F0B159
:1031E0002068806820F001002168886002F0F8FA09
:1031F00005460EE002F0F4FA401B022809D9A06A45
:1032000040F01000A062E06A40F00100E06201209E
:1032100070BD2068806800F001000028EAD100201D
:10322000F6E770B505466C6AA06A00F05000E0B998
:10323000A06A40F40070A0622068806800F46020FA
:10324000B0F5602F0DD1E06858B9A06A20F4807005
:10325000A062A06A00F4805018B9A06A40F0010092
:10326000A062204600F0DEFF03E0206A016B2846E2
:10327000884770BD70B505466C6AA06A40F0400092
:10328000A062E06A40F00400E062204600F0CCFF5B
:1032900070BD70B50446656A284600F0C4FF70BD75
:1032A00038B504460025002000902068806800F0B2
:1032B000010080BB2068806840F0010021688860C0
:1032C000164800681649B0FBF1F0009002E0009843
:1032D000401E009000980028F9D102F081FA0546BE
:1032E00013E002F07DFA401B02280ED9A06A40F0DC
:1032F0001000A062E06A40F00100E06200BF002020
:1033000084F8240000BF012038BD2068806800F0E8
:1033100001000028E5D00020F6E7000000000020B2
:1033200040420F0010B5044800F04AFE0222034953
:10333000014801F06BF810BDEC00002004000020F3
:1033400000BFFEE700B58BB000200690079001207B
:1033500008904FF440400190002002904FF45140FB
:1033600003904FF6FF700490002005900120099013
:1033700001A9154801F00AF920B140F2931113A0F8
:1033800004F0DEFD01200690002007900120089047
:103390004FF440400190002002904FF451400390C0
:1033A0004FF6FF700490002005900120099001A9BC
:1033B000054801F0EBF820B14FF4D47103A004F0FC
:1033C000BFFD0BB000BD0000B02F00202E2E2F53EC
:1033D00072632F63616E2E63000000002DE9F041DF
:1033E00004460D46002700260DB9666B00E0A66B6B
:1033F000206800F5D87000EB0510006800F00400AC
:10340000B060B06858B9206800F5D87000EB0510BE
:10341000006840F2FF7101EA505030600AE0206815
:1034200000F5D87000EB051000686FF0604101EA0C
:10343000D0007060206800F5D87000EB05100068BF
:1034400000F00200F060206800F5D87000EB051075
:10345000406800F00F0030613562206800F5D870D8
:1034600000EB05104068C0F30720F061206800F50C
:10347000D87000EB051080683075206800F5D870B2
:1034800000EB05108068010A7175206800F5D8709E
:1034900000EB05108068010CB175206800F5D8704C
:1034A00000EB05108068000EF075206800F5D870FC
:1034B00000EB0510C0683076206800F5D87000EB8E
:1034C0000510C068010A7176206800F5D87000EB1D
:1034D0000510C068010CB176206800F5D87000EBCB
:1034E0000510C068000EF0764DB920202168C86034
:1034F0002068406920F00A002168486108E0202027
:10350000216808612068406920F050002168486106
:1035100094F83C70222F01D0322F05D120684069E9
:1035200020F40F4021684861CDB994F83C0042284E
:1035300004D0622806D072280CD107E0122084F84B
:103540003C000BE0322084F83C0007E0522084F875
:103550003C0003E0012084F83C0000BF19E094F82F
:103560003C00522804D0622806D072280CD107E013
:10357000122084F83C000BE0222084F83C0007E095
:10358000422084F83C0003E0012084F83C0000BFA6
:1035900000BF204601F0BEFA0020BDE8F081000027
:1035A000002037E0002100EB40021C4B23F83210D2
:1035B0004FF4007100EB400203EBC2025180002186
:1035C00000EB400203EBC202918000EB400203EBF0
:1035D000C202D18000EB400203EBC202118100EB7A
:1035E000400203EBC20291720D4901EB402100EB56
:1035F000400203EBC202D160002100EB400203EB6A
:10360000C2021161012100EB400203EBC2021175FD
:10361000411CC8B21628C5DB70470000A02D002051
:10362000A00100202DE9F34F83B0054628890B281F
:103630007EDB0021284604F0DDFC00907E490098E6
:1036400008700121284604F0D5FC82467A4981F8A9
:1036500001A0009855286CD1BAF1AA0FFBD1288897
:10366000000A88702878C8700221284604F0C2FC3D
:10367000064671490E71112E03D0162E01D00C2E64
:103680007ED10321284604F0B5FC80466A4880F8C4
:1036900005800521284604F0ADFC83460421284618
:1036A00004F0A8FC0BEB00201FFA80F94FEA192068
:1036B0006149887181F807900521284604F09AFC39
:1036C0000446A8EB040002287DD1298908F10900ED
:1036D000814217DA287D012804D102F081F828619F
:1036E0000020287502F07CF82969411A049881426B
:1036F00005D9297A284604F039FC0120287505B03F
:10370000BDE8F08F0120287500270EE0B81DC1B27A
:10371000284604F06FFC4949C8550846C15D07F1C9
:103720000800454A1154781C87B2A742EEDB01E03D
:1037300080E07BE0A01DC1B2284604F05BFC4FEAAC
:10374000006BE01DC1B2284604F054FC0BEB004BAB
:1037500004F10800C1B2284604F04CFC0BEB002B2E
:1037600004F10900C1B2284604F044FC0BEB00014F
:10377000019104F10801304800F046F9029000E0A0
:103780004FE0DDE90110081A41D128882B4B4A4649
:10379000314600F00DFAA01DC1B2284604F02AFC03
:1037A00004F10801244A5054E01DC1B2284604F037
:1037B00021FC04F10901204A5054481EC1B2284698
:1037C00004F018FC00E027E004F10A011A4A505402
:1037D000481EC1B2284604F00DFC04F10B01164A44
:1037E0005054F02104F10C001154401CC2B2124993
:1037F000134803F0D3FE08F10900C1B2284604F0D3
:10380000B5FB4FF400510F4801F0E0FF77E70121CD
:10381000284604F0ABFB0DE00121284604F0A6FB8E
:1038200008E00121284604F0A1FB03E0012128461D
:1038300004F09CFB00BF62E773410020744000204D
:1038400048000020000C014030B50A4600211CE071
:103850000F4B5B6B14335B5C8588C468635583884E
:103860005B1C9BB283804488A34201DB00238380DE
:1038700003895B1C9BB203814488A34203DD438818
:103880000381012383724B1CD9B29142E0DB30BD2E
:10389000B02F00202DE9F0478246884614463E4866
:1038A0000078022801D1BDE8F087002C72DD2046A7
:1038B000E11704EB5171C910A4EBC1018FB237B904
:1038C0000827E11704EB5171C1F3CF0907E0204647
:1038D000E11704EB5171C910491C1FFA81F92F48F7
:1038E000006BC0F800A000202C49096BC8602B4970
:1038F000096B886000261BE008202849096B0861D5
:1039000000250AE0082000FB065018F800102348A4
:10391000006B14304155681C85B2082DF2DB0A217A
:103920001E4801F03DF908B102F09EFF701C86B2FE
:10393000A9F10100B042DFDC1848006B07610025E7
:103940000AE0082000FB065018F800101348006B2E
:1039500014304155681C85B2BD42F2DB0A210F4884
:1039600001F01EF998B10C48007878B902200A4994
:103970000870642001F01AFC01221021084801F0AF
:1039800029FF01224021064801F024FF02E0012026
:103990000149087000BF86E79C000020B02F00207E
:1039A0000008014010B504462068406920F001007D
:1039B0002168486194F83C00122805D120684069CC
:1039C00020F40F402168486194F83C00422804D05C
:1039D000522806D072280CD107E0222084F83C003F
:1039E0000BE0322084F83C0007E0622084F83C00C1
:1039F00003E0012084F83C0000BF00BF204601F036
:103A000027FA002010BD0000F0B502460B46002545
:103A1000681E00210FE0565C7040002407E0060E8F
:103A2000064F57F8265000026840661CB4B2042CBA
:103A3000F5DB4E1CB1B29942EDDBF0BDF885000814
:103A4000F0B58DB006460F461546002404E0305D03
:103A50000BA90855601CC4B2082CF8DB002406E052
:103A600020460830305C09A90855601CC4B2042CFB
:103A7000F6DB002405E0FF21201D09AA1154601C7B
:103A8000C4B2042CF7DB07AB002239460BA804F0C4
:103A900007FB05AB0022394609A804F001FB00240E
:103AA00005E007A8005D01A90855601CC4B2082CF8
:103AB000F7DB002407E005A8015D01AA20460830D5
:103AC0001154601CC4B2082CF5DB00241CE001A8D2
:103AD000005D01AA211D515C4840285501A9201D07
:103AE000085C21460831515C4840211D685401A9F9
:103AF00020460830085C21460C31515C4840214684
:103B000008316854601CC4B2042CE0DB0DB0F0BD79
:103B10003EB5144A14491548FFF792FF002416E0F9
:103B2000A000C01C0F49085C0106A000801C0D4AC3
:103B3000105C01EB0041A000401C105C01EB002078
:103B400012F8241008444DF82400601CC4B2032C61
:103B5000E6DB00F02FF80C226946054800F0C2F9B8
:103B60003EBD0000C0450020F8890008B445002093
:103B700000F4000810B5024801F0C4F910BD0000BF
:103B80001C01002030B590F840500124AC40C56BBA
:103B90006C60046863604468102C04D10468A260FF
:103BA0000468E16003E00468A1600468E26030BD7D
:103BB0007047704708B500200B4908600B488860C3
:103BC0000120C86001F0C0FB00BF34200849C86074
:103BD00000BF6946044801F0FDFA01F053FB642080
:103BE00001F0E4FA08BD0000A445002000F400083C
:103BF0000020024038B504466946204601F0EAFA42
:103C000008B1012038BD0020FCE7000010B50024F9
:103C1000002026490860264888600120C8600121EC
:103C2000234800F087F82349087001212048001D2F
:103C300000F080F82049086001211D48083000F09C
:103C400079F81E490860012119480C3000F072F81B
:103C50001B49086017480078FF2804D10120154946
:103C60000870601CC4B214480068401C28B94FF4A6
:103C7000614011490860601CC4B210480068401CD3
:103C800028B94FF416500D490860601CC4B20C48A6
:103C90000068401C20B9FA2009490860601CC4B2C1
:103CA000002C02DD024800F043F910BDCC45002095
:103CB000002C00089C000020A0000020A400002090
:103CC000A80000200021074AD1610749096941F095
:103CD0000401054A11611146096941F04001116171
:103CE00070470000E0450020002002400021074A04
:103CF000D1610749096941F00201054A1161114684
:103D00004861096941F0400111617047E0450020B8
:103D1000002002400022054BDA61054A126942F098
:103D20000102034B1A61018070470000E04500204A
:103D30000020024010B50246002005E01368064C42
:103D40002360121D431C98B2884202DA034B9A4248
:103D5000F4D90148006810BDC8000020FB2F0008FE
:103D600038B504466946204601F034FA08B101200E
:103D700038BD0020FCE70000002007490860074824
:103D800088600220C86000200549086005488860F6
:103D90003420C860704700009046002000280008CA
:103DA00080460020003000082DE9F04104460E4610
:103DB0001746002501F0C8FA00BF0EE056F825C0EE
:103DC000624600232146022001F066FA08B9241D4C
:103DD00002E00120BDE8F0816D1CBD4202D2034823
:103DE0008442EBD901F04EFA0020F3E7FBFF000814
:103DF00000201E49C96801F0100139B11C49C96988
:103E000041F002011A4AD16140F010001749C96817
:103E100001F0040139B11649C96941F00101144AA0
:103E2000D16140F004001149C96901F0010169B193
:103E30000F49C96941F004010D4AD16100BF0B4926
:103E4000C96921F00101094AD16100BF00BF40F2F8
:103E50000111884206D10549C96921F00101034ACF
:103E6000D16101E00149C86000BF704700200240F5
:103E7000E045002070B5044601F0B2FC054609E0BB
:103E8000601C38B124B101F0ABFC401BA04201D949
:103E9000032070BD1248C06800F001000028EFD177
:103EA0000F48C06800F0200020B100BF20200C495E
:103EB000C86000BF0A48C06800F0100048B9084850
:103EC000C06900F0010020B90548C06800F0040096
:103ED00018B1FFF78DFF0120DBE70020D9E70000D4
:103EE000002002402DE9F04104460E461746002509
:103EF00001F02AFA00BF0FE056F825C06246002301
:103F00002146022001F0C8F908B9241D03E001F0A0
:103F1000B9F9BDE8F0816D1CBD4202D2034884426C
:103F2000EAD901F0AFF900BFF3E70000FBF70008A2
:103F30002DE9FF410446002501F006FA00BF3420B8
:103F40001849C86000BF1848FFF754FEC82001F0A8
:103F50002DF9042615480078009015480068019056
:103F600014480068029014480068039000BF0FE0F6
:103F70005DF825703A4600232146022001F08CF9B5
:103F800008B9241D03E0012004B0BDE8F0816D1CD8
:103F9000B54202D209488442EAD901F073F90020FF
:103FA000F2E7000000200240CC4500209C000020E9
:103FB000A0000020A4000020A8000020FB2F000883
:103FC000F8B5044600260020009000BF94F82400B5
:103FD000012801D10220F8BD012084F8240000BF8F
:103FE0002046FFF7F5F80646002E62D1A06A20F4BD
:103FF000885040F00200A062022001F043FD3049E9
:104000000968B1FBF0F04000009002E00098401E0B
:10401000009000980028F9D12046FFF741F9206868
:10402000806840F008002168886001F0D9FB0546EF
:1040300011E001F0D5FB401B0A280CD9A06A20F042
:10404000020040F01000A06200BF002084F82400AD
:1040500000BF0120BFE72068806800F0080000284A
:10406000E7D12068806840F004002168886001F092
:10407000B7FB054611E001F0B3FB401B0A280CD941
:10408000A06A20F0020040F01000A06200BF0020F3
:1040900084F8240000BF01209DE72068806800F0BC
:1040A00004000028E7D1A06A20F0020040F00100DF
:1040B000A06200BF002084F8240000BF30468AE7D9
:1040C0000000002038B5024600230020009000BF09
:1040D00092F82400012801D1022038BD012082F885
:1040E000240000BF4868072812D21068406B0C7982
:1040F000641E04EB84051F24AC40A0430D796D1EA3
:1041000005EB85050C68AC4020431468606327E02C
:1041100048680D2812D21068006B0C79E41F04EB7C
:1041200084051F24AC40A0430D79ED1F05EB8505E8
:104130000C68AC4020431468206311E01068C06A2A
:104140000C790D3C04EB84051F24AC40A0430D7991
:104150000D3D05EB85050C68AC4020431468E0621A
:1041600008680A2812D31068C0680C780A3C04EB6F
:1041700044050724AC40A0430D780A3D05EB4505F6
:104180008C68AC4020431468E0600FE01068006960
:104190000C7804EB44050724AC40A0430D7805EBF4
:1041A00045058C68AC4020431468206108681028DD
:1041B00002D00868112827D1174C1068A0421ED1E0
:1041C0001068806800F40000F0B91068806840F45E
:1041D00000001468A0600868102815D10F48006816
:1041E0000F4CB0FBF4F000EB80004000009002E0C8
:1041F0000098401E009000980028F9D104E0906AD1
:1042000040F020009062012300BF002082F82400CB
:1042100000BF184661E700000024014000000020B4
:1042200040420F0070477047704700002DE9F04191
:104230000446002700250026A84614B90120BDE841
:10424000F081A06810B1606900B100BFA06A30B908
:104250000020E06284F82400204600F089F820461F
:10426000FEF7B6FF0746A06A00F01000002873D1E1
:10427000002F71D1A06A20F4885040F00200A062A3
:10428000E16960680843E16840EA41000643A068CC
:10429000B0F5807F02D0A068012802D14FF4807071
:1042A00000E0002005436069012811D1E06838B9B9
:1042B000A069401E4FF4006141EA4030054307E029
:1042C000A06A40F02000A062E06A40F00100E062D5
:1042D0002068406820F469402843216848602068CD
:1042E000806821490840304321688860A068B0F5A3
:1042F000807F02D0A068012802D14FF4807000E0D6
:104300000020B0F5807F03D1208A401E4FEA00587C
:104310002068C06A20F4700040EA08002168C86282
:104320002068806811490840B04208D10020E0624E
:10433000A06A20F0020040F00100A06211E0A06A33
:1043400020F0020040F01000A062E06A40F001009E
:10435000E062012705E0FFE7A06A40F01000A062DC
:10436000012738466BE70000FDF7E1FFFE0E1FFF57
:1043700010B586B004461C492068884232D100BF7F
:104380001A48806940F400701849886108468069BD
:1043900000F40070019000BF00BF03200290039062
:1043A00002A9134801F084F812481349086000205C
:1043B00048600021104881608021C160490001618E
:1043C00089004161202181610021C16100F068FE06
:1043D00018B17E2109A003F0B3FD00BF064820629A
:1043E000446200BF06B010BD00240140001002402E
:1043F00000080140080002401C0100202E2E2F530F
:1044000072632F6164632E63000000002DE9F041A8
:1044100004460D461646002757492068884203D0B7
:1044200056492068884205D15348001D006800F4B1
:10443000702000E0002000287ED100BF94F8240006
:10444000012802D10220BDE8F081012084F8240077
:1044500000BF2046FEF724FF0746002F6DD1A06A5B
:1044600040F60161884340F48070A06243492068AF
:10447000884209D14048001D006800F4702008B946
:10448000012002E0002000E0012078B1A06A20F4C1
:104490008010A0622068406800F4806000B3A06AC9
:1044A00020F4005040F48050A06219E0A06A40F46B
:1044B0008010A06230492068884203D02F492068CC
:1044C000884205D12C48001D006800F4806000E09F
:1044D000002028B1A06A20F4005040F48050A0626F
:1044E000A06A00F4805020B1E06A20F00600E0628B
:1044F00001E00020E06200BF002084F8240000BF3B
:104500001F48216A88621F48216AC8621E48216AC2
:1045100008636FF00200216808602068806840F43A
:10452000807021688860226802F14C0133462A4677
:10453000206A00F0EDFD01E01AE014E020688068D8
:1045400000F46020B0F5602F06D12068806840F448
:10455000A000216888600CE02068806840F480102A
:104560002168886005E000BF002084F8240000E096
:104570000127384667E70000002401400028014079
:1045800023320008933200087532000830B5024625
:1045900000230C7D012000FA04F31068D0F800021B
:1045A00020F47C5001254C6A45EA04242043146819
:1045B000C4F800021068D0F81C0298431468C4F8CC
:1045C0001C02C869E8B91068D0F80C029843146856
:1045D000C4F80C02888880B28C8940EA04441068D0
:1045E00000F510704D6940F83540088880B20C899C
:1045F00040EA0444106800F510704D6900EBC500F6
:104600004460C86901281DD11068D0F80C02184315
:104610001468C4F80C02888880B20C8840EA04440C
:10462000106800F510704D6940F83540888980B2F7
:104630000C8940EA0444106800F510704D6900EBE5
:10464000C5004460886938B91068D0F804029843FE
:104650001468C4F8040206E01068D0F80402184395
:104660001468C4F80402086938B91068D0F8140254
:1046700098431468C4F8140206E01068D0F81402D5
:1046800018431468C4F81402086A012806D1106897
:10469000D0F81C0218431468C4F81C021068D0F843
:1046A000000220F001001468C4F80002002030BDB0
:1046B000704700002DE9F041044600250026002740
:1046C000A8462068C068C0F3001520684069C0F3A0
:1046D000C0062DB126B148F4007810202168C860CA
:1046E00020680069C0F3001520684069C0F3801697
:1046F0002DB126B148F48068102021680861206837
:10470000406900F0010000283BD0206880687A49A9
:104710000840884201D1012000E0002005462068C1
:10472000806876490840884201D1012000E00020DD
:1047300006462068806872490840884201D10120FD
:1047400000E0002007460DB906B9D7B1206880689F
:10475000C0F3400520688068C0F340262068806868
:1047600000F001070DB906B91FB12046FFF71AF98D
:1047700001E048F4006820688068624908432168C5
:1047800088602068C06800F0030520684069C0F3B5
:10479000400625B11EB100212046FEF71FFE20680D
:1047A000006900F0030520684069C0F3001625B1D8
:1047B0001EB101212046FEF711FE206C40EA0800E0
:1047C00020642068806900F0010520684069C0F31A
:1047D000002620684069C0F3C0372DB126B11FB153
:1047E000206C40F00100206420688069C0F340051F
:1047F00020684069C0F3402620684069C0F3C03794
:104800002DB126B11FB1206C40F002002064206859
:104810008069C0F3800520684069C0F38026206865
:104820004069C0F3C0372DB126B11FB1206C40F0F4
:10483000040020642068806900F0700008B901203D
:1048400000E00020054620684069C0F3C0262068CB
:104850004069C0F3C03795BB8EB387B320688069C9
:1048600000F07005402D1BD006DC102D09D0202D46
:104870000CD0302D24D10EE0502D16D0602D1FD13C
:1048800018E0206C40F0080020641AE0206C40F032
:104890001000206415E0206C40F02000206410E03F
:1048A000206C40F0400020640BE0206C40F0800061
:1048B000206406E0206C40F48070206401E007E092
:1048C00000BF00BF2068806920F070002168886107
:1048D000206C78B1042021684860012084F83C00F5
:1048E0002068406948F65B7188432168486120462A
:1048F000FFF7DEFEBDE8F0810100000400010008C2
:1049000000000110090501002DE9F04104460027CF
:104910000026002514B90120BDE8F08194F83C0080
:1049200028B9002084F83D00204600F0A5F80220B8
:1049300084F83C002068006820F0020021680860CC
:104940002068006840F001002168086000F048FF1E
:1049500006460EE000F044FF801B0A2809D9032018
:1049600084F83C0000BF002084F83D0000BF032015
:10497000D2E72068406800F001000028EAD02068F3
:10498000406800F00100002867D0A069012802D12A
:1049900045F0800501E025F08005E069012802D19D
:1049A00045F0400501E025F04005206A012802D1CC
:1049B00045F0200501E025F02005606A012802D1BC
:1049C00045F0100501E025F01005A06A012802D18C
:1049D00045F0080501E025F00805E06A012802D14C
:1049E00045F0040501E025F004052068006820F08A
:1049F000FC00284321680860D4E9020108432169CA
:104A00000843616908436168491E08432168C86119
:104A10002068006820F001002168086000F0E0FED6
:104A200006460EE000F0DCFE801B0A2809D90320B0
:104A300084F83C0000BF002084F83D0000BF032044
:104A40006AE72068406800F001000028EAD1206889
:104A5000406800F0010000B90127012F06D10020B5
:104A60002064012084F83C00002055E7042084F8ED
:104A70003C00012050E7000010B586B004461F49F5
:104A80002068884237D100BF1D48C06940F00070DF
:104A90001B49C8610846C06900F00070019000BF62
:104AA00000BFC814029000200390049002A915488A
:104AB00000F0FEFC4FF4805002900220039003208F
:104AC000059002A90F4800F0F3FC002211461420C3
:104AD00000F063FF142000F053FF0B4820630B48E5
:104AE0006063FEF72FFC0A480068406940F002004E
:104AF00007490968486106B010BD00000064004025
:104B00000010024000080140600100207C010020EC
:104B1000B02F002070B50446606B806810B9606BE0
:104B2000006940B91A480068406940F0020018491D
:104B30000968486170BD00251DE0606B006815497B
:104B400031F81510884214D1606B008805EB4501DF
:104B5000114A22F83100626B117C05EB45020E4BC5
:104B600003EBC200FEF770FE00F03AFE0B4908604E
:104B700003E0681C85B2162DDFDB00BF0448006827
:104B8000406940F0020002490968486100BFD1E76E
:104B9000B02F0020CC830008A02D0020940000201E
:104BA0002DE9F04104460E46042500272068806860
:104BB00000F08060B0F1806F0DD02068806800F058
:104BC0000060B0F1006F06D02068806800F080506F
:104BD000B0F1805F7ED100BF94F83D00012802D182
:104BE0000220BDE8F081012084F83D0000BF94F868
:104BF0003C00222804D0322806D062280CD107E0DD
:104C0000422084F83C000BE0522084F83C0007E08E
:104C1000722084F83C0003E0122084F83C0000BFBE
:104C200000BF2068806800F0806008B1002507E0C0
:104C30002068806800F0006008B1012500E00225CE
:104C4000206800F5C07000EB0510006800F001015D
:104C5000206800F5C07000EB05100160206B8068D3
:104C600098B9206800F5C07000EB05100068216B52
:104C7000C968226B128841EA42510843216801F554
:104C8000C07101EB0511086015E0206800F5C070E7
:104C900000EB05100068216B8968226B526841EABD
:104CA000C201226BD26811430143206800F5C07035
:104CB00000EB05100160206B007C00F00F00216B01
:104CC0000861206800F5C07000EB0510406820F016
:104CD0000F0100E0B1E0206800F5C07000EB0510A6
:104CE0004160206800F5C07000EB05104068216B42
:104CF00009690843216801F5C07101EB051148609D
:104D0000206BC07D0106206B807D41EA0041206B55
:104D1000407D41EA0020216B097D0843216801F5AF
:104D2000C07101EB05118860206BC07E0106206B0D
:104D3000807E41EA0041206B407E41EA0021206BE9
:104D4000007E0143206800F5C07000EB0510C160D3
:104D5000206800F5C07000EB0510006840F001010C
:104D6000206800F5C07000EB0510016000F038FD10
:104D7000074620E0701CF0B126B100F031FDC01BE9
:104D8000B04218D9032084F83C001DB98020216866
:104D9000886009E0012D03D1E8032168886003E001
:104DA0004FF400002168886000BF002084F83D00B7
:104DB00000BF032015E74DB92068806821490840ED
:104DC000884201D1012016E0002014E0012D09D114
:104DD000206880681C490840884201D101200AE00F
:104DE000002008E02068806818490840884201D106
:104DF000012000E000200028BCD094F83C004228AC
:104E000004D0522806D072280CD107E0222084F862
:104E10003C000BE0322084F83C0007E0622084F87C
:104E20003C0003E0012084F83C0000BF00BF00BF4D
:104E3000002084F83D0000BFD3E6042084F83C0045
:104E40000120CEE60100000400010008000001106E
:104E50007047000070B50446002594F82100022830
:104E600003D00420A063012548E02068006820F0FA
:104E70000E00216808602068006820F001002168A9
:104E800008601F492068884201D1012026E01C49A2
:104E900014312068884201D110201FE018492831C0
:104EA0002068884201D1801518E015493C312068FE
:104EB000884201D1801411E01149503120688842A4
:104EC00002D14FF4803009E00D49643120688842F6
:104ED00002D14FF4801001E04FF08070084908398A
:104EE0004860012084F8210000BF002084F82000E1
:104EF00000BF606B10B12046616B8847284670BDCB
:104F00000800024070B50446E06B0568206806683A
:104F100094F84010042088402840002846D006F02D
:104F20000400002842D02068006800F0200028B962
:104F30002068006820F00400216808605749206854
:104F4000884201D1042027E0544914312068884266
:104F500001D1402020E0514928312068884201D108
:104F6000001519E04D493C312068884202D14FF4C8
:104F7000804011E0494950312068884202D14FF405
:104F8000802009E0454964312068884202D14FF40D
:104F9000800001E04FF08060404908394860E06AD5
:104FA00000287AD02046E16A884776E094F84010DD
:104FB000022088402840A0B306F0020088B3206891
:104FC000006800F0200040B92068006820F00A0066
:104FD00021680860012084F8210030492068884257
:104FE00001D1022028E02D4914312068884201D1E6
:104FF000202021E0294928312068884201D140152C
:105000001AE026493C312068884202D14FF4005012
:1050100012E0224950312068884203D14FF4003019
:105020000AE017E01D4964312068884202D14FF43C
:10503000001001E04FF0007018490839486000BFC7
:10504000002084F8200000BFA06A30B32046A16A87
:10505000884722E094F84010082088402840E0B1BA
:1050600006F00800C8B12068006820F00E00216832
:10507000086094F8401001208840E16B48600120EE
:10508000A06384F8210000BF002084F8200000BF46
:10509000206B10B12046216B884770BD080002408C
:1050A0000146002209B901207047184B0868C01A50
:1050B0001423B0FBF3F08000086414480838C86378
:1050C000022081F821000868026843F6F0708243EC
:1050D000D1E901031843CB6818430B6918434B69A6
:1050E00018438B691843CB69184302430868026070
:1050F00000208862C862086348638863012081F8E1
:105100002100002081F8200000BFCDE70800024008
:105110002DE9F04104460D4616461F464FF00008A3
:1051200000BF94F82000012802D10220BDE8F081E0
:10513000012084F8200000BF94F8210001282CD120
:10514000022084F821000020A0632068006820F07D
:105150000100216808603B46324629462046FEF79A
:1051600011FDE06A30B12068006840F00E0021684F
:1051700008600BE02068006820F0040021680860E7
:105180002068006840F00A00216808602068006814
:1051900040F001002168086006E000BF002084F8AC
:1051A000200000BF4FF002084046BFE770B504463C
:1051B00000F016FB06462546681C10B1044800782E
:1051C000054400BF00F00CFB801BA842FAD370BD61
:1051D000D40000202DE9F04104460E4601270025A9
:1051E00000BF2648007E012802D10220BDE8F081E0
:1051F00001202249087600BF2068022813D14CF212
:105200005030FEF737FE90BB0120FEF75BFD4CF2FD
:105210005030FEF72FFE07461948006920F00400C1
:105220001749086123E04CF25030FEF723FEF0B935
:105230004FF0FF303060A56812E02846FEF756FDBB
:105240004CF25030FEF716FE07460D48006920F07C
:1052500002000B4908610FB1356007E005F5806574
:10526000D4E9021001EB8020A842E6D800BF00BFBD
:1052700000200249087600BF3846B7E7E045002025
:10528000002002400348006940F0800001490861A5
:1052900000207047002002402DE9FE4F05468B4656
:1052A00017469846012600240020029000BF24489B
:1052B000007E012802D10220BDE8FE8F0120204996
:1052C000087600BF4CF25030FEF7D4FD064686BB90
:1052D000012D02D10120029006E0022D02D1022010
:1052E000029001E00420029000241EE02201B94651
:1052F000C24648465146FDF715FF80B20190022094
:1053000000FB04B000900199FEF704FD4CF2503010
:10531000FEF7B0FD06460B48006920F00100094980
:10532000086106B104E0601CC4B202988442DDDB6F
:1053300000BF00BF00200249087600BF3046BBE72F
:10534000E04500200020024000200849096901F0E2
:10535000800151B10649054A516006495160114624
:10536000096901F0800101B101207047002002406D
:1053700023016745AB89EFCD2DE9F04102460B468D
:1053800000200021002400267FE00127874007EA53
:105390000301002978D0FF2901D8174600E0171D26
:1053A0003D46FF2901D8870002E0A0F10807BF00B1
:1053B0003E462F684FF00F0C0CFA06FC27EA0C074C
:1053C0004FF0040C0CFA06FC47EA0C072F60D76874
:1053D0008F43D760304F4FEA900C57F82C40870727
:1053E0004FEA177C0F2707FA0CF73C402B4FBA42C5
:1053F00001D100270FE02A4FBA4201D101270AE06C
:10540000284FBA4201D1022705E0274FBA4201D105
:10541000032700E004274FEA807C4FEA1C7C07FA50
:105420000CF7A74230D187074FEA177C0F2707FAFE
:105430000CF4194F4FEA900C57F82C70A743DFF883
:1054400058C04FEA90084CF82870184F3F688F43B7
:10545000DFF858C0CCF800700CF104073F688F43A8
:105460000CF1040CCCF800700CF104073F688F437A
:105470000CF1040CCCF800700CF104073F688F436A
:105480000CF1040CCCF80070401C23FA00F7002F3C
:105490007FF47BAFBDE8F0810800014000080140C7
:1054A000000C0140001001400014014000040140C4
:1054B0002DE9F847034600240020002584460027F4
:1054C00000226EE14FF0010808FA02F4D1F80080E2
:1054D00008EA0400A0427DD1DFF8D0A2D1F8048010
:1054E000A8EB0A09D0453AD014DCB8F1030F50D02C
:1054F00009DCB8F1000F31D0B8F1010F1CD0B8F1C0
:10550000020F49D120E0B8F1110F18D0B8F1120FF5
:1055100042D11EE0B9F5881F25D006DCB9F5803FE1
:1055200020D0B9F5801F37D11AE0B9F5001F18D087
:10553000B9F5041F30D117E0D1F80CC02DE0D1F837
:105540000C8008F1040C28E0D1F80C8008F1080C5C
:1055500023E0D1F80C8008F10C0C1EE000BF00BF66
:1055600000BF00BF00BF00BFD1F80880B8F1000F36
:1055700002D14FF0040C0BE0D1F80880B8F1010F14
:1055800003D14FF0080C1C6102E04FF0080C5C6185
:1055900003E04FF0000C00E000BF00BFFF2801D87F
:1055A000984601E003F104084646FF2802D84FEA76
:1055B000820803E0A2F108084FEA88084746D6F8B7
:1055C00000804FF00F0909FA07F928EA09080CFAD8
:1055D00007F900E088E048EA0908C6F80080D1F839
:1055E000048008F08058B8F1805F7DD100BFDFF8FB
:1055F000C081D8F8188048F00108DFF8B491C9F8E4
:105600001880C846D8F8188008F00108CDF8008046
:1056100000BF00BF4FEAB9384FEA920958F8295045
:105620004FEA82784FEA18794FF00F0808FA09F824
:1056300025EA0805DFF87C81434502D14FF00008D8
:1056400016E0DFF87481434502D14FF001080FE006
:10565000DFF86881434502D14FF0020808E0DFF827
:105660006081434502D14FF0030801E04FF0040888
:105670004FEA82794FEA197908FA09F848EA0505EC
:10568000DFF840814FEA920948F82950D1F80480A8
:1056900008F48038B8F5803F0AD1DFF82C81D8F8BB
:1056A000008048EA0008DFF82091C9F8008009E08E
:1056B000DFF81481D8F8008028EA0008DFF80891A4
:1056C000C9F80080D1F8048008F40038B8F5003F2C
:1056D00010D1DFF8F48008F10408D8F8008048EA17
:1056E0000008DFF8E49000E05AE009F10409C9F885
:1056F00000800DE0DFF8D08008F10408D8F80080C1
:1057000028EA0008DFF8C09009F10409C9F8008010
:10571000D1F8048008F48018B8F5801F0ED1DFF8A6
:10572000A88008F10808D8F8008048EA0008DFF8E7
:10573000989009F10809C9F800800DE0DFF8888029
:1057400008F10808D8F8008028EA0008DFF8789007
:1057500009F10809C9F80080D1F8048008F400189C
:10576000B8F5001F0ED1DFF8608008F10C08D8F8FA
:10577000008048EA0008DFF8509009F10C09C9F8E8
:1057800000800DE0DFF8408008F10C08D8F80080B8
:1057900028EA0008DFF8309009F10C09C9F8008008
:1057A000521C102AFFF48EAEBDE8F88700001110DD
:1057B0000010024000080140000C014000100140B0
:1057C000001401400800014000040140C2684A4042
:1057D000C26070470AB1016101E00B0403617047C8
:1057E0000148006870470000CC00002070B50446F6
:1057F0000CB9012070BD4CF6CC402168086045F220
:10580000555021680860D4E9001048602168A068FC
:105810008860FFF7E5FF054606E0FFF7E1FF401B64
:10582000302801D90320E5E72068C0680028F4D1BA
:105830004AF6AA20216808600020DBE701464AF604
:10584000AA200A6810600020704700000348006822
:10585000034909780844014908607047CC000020DA
:10586000D400002010B50848006840F01000064938
:105870000860032000F0D0F8002000F007F800F0E6
:105880002BF8002010BD00000020024070B5044637
:105890000E4800784FF47A71B1FBF0F00C490968BA
:1058A000B1FBF0F5284600F08CFD08B1012070BD79
:1058B000102C07D200222146501E00F06EF8054839
:1058C000046001E00120F2E70020F0E7D4000020AE
:1058D00000000020D000002008B500BF1F488069EC
:1058E00040F001001D4988610846806900F0010010
:1058F000009000BF00BF032000F08EF80022114688
:105900006FF00B0000F049F8002211466FF00A001A
:1059100000F043F8002211466FF0090000F03DF856
:1059200000221146501F00F038F800221146101FC7
:1059300000F033F800221146901E00F02EF80022ED
:105940001146501E00F029F800BF0549486820F0B4
:10595000E06040F00070486000BF08BD00100240E9
:105960000000014000BF00F01F0201219140034AE6
:10597000430942F8231000BF7047000080E100E0B7
:1059800000BF00F01F02012191404209920002F184
:10599000E022C2F8001100BF70472DE9F05F804699
:1059A0000D461646002701F09FF8074639462A465D
:1059B000334601F00700C0F1070ABAF1040F02D91B
:1059C0004FF0040A01E0C0F1070AD14600F1040AD1
:1059D000BAF1070F02D24FF0000A01E0A0F1030A6A
:1059E000D4464FF0010A0AFA09FAAAF1010A0AEAB2
:1059F000020A0AFA0CFA4FF0010B0BFA0CFBABF19E
:105A0000010B0BEA030B4AEA0B042146404601F066
:105A100073F8BDE8F09F000000BF00F00702064BDE
:105A200019684FF6FF031940044B0B4343EA022168
:105A3000014B196000BF70470CED00E00000FA0553
:105A400000BF00BF00BF00BF00BFBFF34F8F00BF4C
:105A500000BF00BF0948006800F4E060084908433F
:105A6000001D0649086000BF00BF00BFBFF34F8F95
:105A700000BF00BF00BF00BF00BFFDE70CED00E0AE
:105A80000000FA052DE9F04385B006463DA30FCB93
:105A900001AC0FC43FA0006800904FF00008002543
:105AA00000270024A146012E30D0022E58D0102EFF
:105AB00061D139484468006800F0807000B301A8E3
:105AC000C4F38341475C04F4803070B132484068CD
:105AD000C0F340401DF8008004F4803040B12F48EE
:105AE000B0FBF8F000FB07F502E02D4807FB00F5DE
:105AF0002948406800F48000B0F5800F01D1A94624
:105B000003E068000321B0FBF1F935E02248046AA4
:105B100004F44070B0F5807F05D104F0020010B1AC
:105B20004FF400491BE004F44070B0F5007F07D14A
:105B30001948406A00F0020010B149F640490EE0F1
:105B400004F44070B0F5407F07D11348006800F4BA
:105B5000003010B14FF2244901E04FF000090BE092
:105B600000F0A0F90C494968C1F38131491C490092
:105B7000B0FBF1F900E000BF00BF484605B0BDE84A
:105B8000F083000002030405060708090A0B0C0D48
:105B90000E0F1010010200000010024000127A00E7
:105BA00000093D00F8B5044600260025207800F0E5
:105BB000010000286BD000274348C06900F08050E6
:105BC00070B900BF4048C06940F080503E49C8618C
:105BD0000846C06900F08050009000BF00BF012758
:105BE0003A48006800F48070B0B93848006840F462
:105BF000807036490860FFF7F3FD064606E0FFF7C0
:105C0000EFFD801B642801D90320F8BD2F480068F0
:105C100000F480700028F2D02B48006A00F4407530
:105C20002DB3A08800F44070A84220D02648006A16
:105C300020F44075012026490860002008602248B1
:105C4000056205F0010090B1FFF7CAFD064608E0C5
:105C5000FFF7C6FD801B41F28831884201D903203D
:105C6000D3E71948006A00F002000028F0D0164877
:105C7000006A20F440706168084313490862012FEC
:105C800004D10846C06920F08050C86100BF207868
:105C900000F00200022807D10B48406820F4404081
:105CA000A168084308494860207800F010001028D7
:105CB00007D10548406820F48000E16808430249A4
:105CC00048600020A1E70000001002400070004082
:105CD0004004424270B504460D4600266248006802
:105CE00000F00700A8420ED25F48006820F00700CD
:105CF00028435D4908600846006800F00700A84294
:105D000001D0012070BD207800F00200022807D1E8
:105D10005648406820F0F000A168084353494860A5
:105D2000207800F0010000285DD06068012806D1CD
:105D30004E48006800F4003090B90120E2E7606846
:105D4000022806D14948006800F0007040B90120DF
:105D5000D8E74648006800F0020008B90120D1E702
:105D60004248406820F00300616808433F494860AA
:105D7000FFF736FD06466068012810D108E0FFF7FE
:105D80002FFD801B41F28831884201D90320B9E7F9
:105D90003648406800F00C000428F0D123E0606829
:105DA000022810D108E0FFF71BFD801B41F288316B
:105DB000884201D90320A5E72C48406800F00C0078
:105DC0000828F0D10FE008E0FFF70AFD801B41F240
:105DD0008831884201D9032094E72448406800F0C4
:105DE0000C000028F0D12048006800F00700A8420D
:105DF0000ED91D48006820F0070028431A490860A2
:105E00000846006800F00700A84201D0012079E7A9
:105E1000207800F00400042807D11448406820F4DA
:105E2000E060E168084311494860207800F008000C
:105E3000082808D10D48406820F46050216940EAE4
:105E4000C1000A49486000F03DF808494968C1F3BB
:105E50000311074A515CC840064908600020FFF75B
:105E600015FD00204EE70000002002400010024017
:105E7000B48300080000002001480068704700005B
:105E80000000002000B5FFF7F7FF04494968C1F39F
:105E90000221034A515CC84000BD000000100240CE
:105EA000C483000800B5FFF7E7FF04494968C1F360
:105EB000C221034A515CC84000BD000000100240EE
:105EC000C4830008F0B585B00FF26C0C9CE8E010BC
:105ED00001A8A0E8E0101CA52D6800950021002273
:105EE000002300240020194D696801F00C05F5B16C
:105EF000042D02D0082D19D101E0154819E001AD9B
:105F0000C1F38346AC5D01F4803555B10F4D6D682A
:105F1000C5F340451DF805200D4D6543B5FBF2F373
:105F200002E00C4D04FB05F3184602E000BF0848F0
:105F300000BF00BF05B0F0BD020304050607080955
:105F40000A0B0C0D0E0F1010010200000010024091
:105F500000127A0000093D00F8B5044600252078BB
:105F600000F00100002878D0F848406800F00C00EC
:105F700004280CD0F548406800F00C00082811D126
:105F8000F248406800F48030B0F5803F0AD1EF4815
:105F9000006800F4003000285FD0606800285CD101
:105FA0000120F8BD00BF6068B0F5803F06D1E7482A
:105FB000006840F48030E549086028E0606858B91E
:105FC000E248006820F48030E04908600846006834
:105FD00020F4802008601AE06068B0F5A02F0BD193
:105FE000DA48006840F48020D84908600846006814
:105FF00040F4803008600AE0D448006820F4803023
:10600000D24908600846006820F48020086000BF7C
:10601000606888B1FFF7E4FB054606E0FFF7E0FBA8
:10602000401B642801D90320BBE7C848006800F47E
:1060300000300028F2D010E0FFF7D2FB054606E062
:10604000FFF7CEFB401B642801D90320A9E7BF4816
:10605000006800F400300028F2D1207800F002003F
:10606000022857D1B948406800F00C0050B1B74839
:10607000406800F00C00082818D1B448406800F4CB
:10608000803098B9B148006800F0020020B1206962
:10609000012801D0012084E7AC48006820F0F80016
:1060A000616940EAC100A949086033E02069E8B1AC
:1060B0000120A7490860FFF793FB054606E0FFF7BC
:1060C0008FFB401B022801D903206AE79F48006824
:1060D00000F002000028F2D09C48006820F0F80090
:1060E000616940EAC1009949086013E000209849BD
:1060F0000860FFF775FB054606E0FFF771FB401BE4
:10610000022801D903204CE79048006800F0020003
:106110000028F2D1207800F0080008282DD1A069CD
:10612000B8B101208B490860FFF75AFB054606E02D
:10613000FFF756FB401B022801D9032031E78348B3
:10614000406A00F002000028F2D0012000F018FDA3
:1061500013E000207F490860FFF742FB054606E098
:10616000FFF73EFB401B022801D9032019E77748BF
:10617000406A00F002000028F2D1207800F004000C
:10618000042873D100267148C06900F0805070B9AE
:1061900000BF6E48C06940F080506C49C861084635
:1061A000C06900F08050009000BF00BF01266A481F
:1061B000006800F48070B0B96748006840F48070EF
:1061C00065490860FFF70CFB054606E0FFF708FB92
:1061D000401B642801D90320E3E65F48006800F40F
:1061E00080700028F2D000BFE068012806D157482F
:1061F000006A40F001005549086227E0E06858B99C
:106200005248006A20F00100504908620846006ABE
:1062100020F00400086219E0E06805280BD14B4823
:10622000006A40F00400494908620846006A40F0EC
:10623000010008620AE04548006A20F00100434975
:1062400008620846006A20F00400086200BFE068A7
:10625000A0B1FFF7C5FA054609E0FFF7C1FA401BF8
:1062600041F28831884202D903209AE622E0374879
:10627000006A00F002000028EFD012E0FFF7B0FA49
:10628000054608E0FFF7ACFA401B41F2883188422E
:1062900001D9032085E62D48006A00F0020000289D
:1062A000F0D1012E05D12948C06920F0805027493E
:1062B000C86100BFE069C8B32448406800F00C0022
:1062C000082860D0E069022848D1002020490866EB
:1062D000FFF786FA054606E0FFF782FA401B022820
:1062E00001D903205DE61948006800F0007000281D
:1062F000F2D1206AB0F5803F07D11448406820F4FD
:106300000030A168084311494860D4E908010843F6
:106310000E49496821F4741108430C494860012072
:106320000B490866FFF75CFA054607E02DE0FFF72A
:1063300057FA401B022801D9032032E603480068BF
:1063400000F000700028F2D01FE0000000100240B2
:1063500000004242800442420070004000200C498C
:106360000866FFF73DFA054606E0FFF739FA401BDD
:10637000022801D9032014E60648006800F00070E6
:106380000028F2D101E001200BE6002009E6000020
:106390000000424200100240042808D14FF0E021E2
:1063A000096941F004014FF0E022116107E04FF06C
:1063B000E021096921F004014FF0E02211617047EA
:1063C000704770B504462546681EB0F1807F01D342
:1063D00001200FE0681E4FF0E02148610F214FF0CF
:1063E000FF3000F089FB00204FF0E021886107209A
:1063F0000861002070BD10B5FFF7E2FF10BD10B5B9
:1064000004460CB9012010BD242084F83900204630
:1064100000F0EEF80020E06384F8390084F83A00D8
:1064200000BF84F8380000BF00BFECE770470000F1
:106430002DE9F0470446206805682068C668206892
:1064400047694FF00008C14605F00F08B8F1000F8A
:106450000AD105F0200038B106F0200020B1204616
:1064600001F049F8BDE8F087B8F1000F6DD007F0F2
:10647000010018B906F49070002866D005F00100FC
:1064800030B106F4807018B1E06B40F00100E063B9
:1064900005F0040030B107F0010018B1E06B40F0E6
:1064A0000200E06305F0020030B107F0010018B10E
:1064B000E06B40F00400E06305F0080030B107F045
:1064C000010018B1E06B40F00800E063E06B68B3D6
:1064D00005F0200028B106F0200010B1204601F0A0
:1064E0000AF820684069C0F38019E06B00F00800EA
:1064F00010B9B9F1000F22D0204600F08DFF2068BE
:10650000406900F04000B0B12068406920F04000D0
:1065100021684861606B50B11748616B4863606BDC
:10652000FEF798FC10B1606B416B88470CE0204689
:10653000FFF77CFF08E02046FFF778FF04E02046E5
:10654000FFF774FF0020E0638CE705F0800030B1B6
:1065500006F0800018B1204601F0F2F982E705F05C
:10656000400030B106F0400018B1204600F064FF52
:1065700078E700BF76E700008173000810B5044695
:106580000CB9012010BDA06900B100E000BF94F873
:10659000390028B9002084F83800204600F05AF865
:1065A000242084F839002068C06820F40050216855
:1065B000C860204601F086F82068006920F4904009
:1065C000216808612068406920F02A00216848613C
:1065D0002068C06840F400502168C8600020E06373
:1065E000202084F8390084F83A000020CAE700002F
:1065F00010B504461249206888420ED11148C0697E
:1066000020F480200F49C8614FF440610E48FEF726
:10661000B3FE2720FFF7A6F911E00C492068884255
:106620000DD10848806920F48040064988614FF404
:10663000C0610748FEF7A0FE2520FFF793F910BDC3
:106640000048004000100240000C014000380140AA
:106650000008014010B586B004464B4920688842C6
:1066600042D100BF4948C06940F480204749C86111
:106670000846C06900F48020019000BF00BF0815E3
:106680000290022003900320059002A94048FEF7E3
:106690000FFF4FF40060029000200390049002A9C5
:1066A0003B48FEF705FF002211462720FFF775F94A
:1066B0002720FFF765F937480068C06840F480700C
:1066C00034490968C86033480068406940F00100F7
:1066D0003049096848612F480068C06840F02000D0
:1066E0002C490968C8604CE02B492068884248D191
:1066F00000BF2648806940F48040244988610846EC
:10670000806900F48040019000BF00BF00BF0846D0
:10671000806940F0040088610846806900F0040048
:10672000019000BF00BF4815029002200390032093
:10673000059002A91948FEF7BBFE4FF48060029055
:1067400000200390049002A91448FEF7B1FE002235
:1067500011462520FFF721F92520FFF711F92068C0
:10676000C06840F480702168C8602068406940F0CB
:106770000100216848612068C06840F0200021685D
:10678000C86006B010BD0000004800400010024084
:10679000000C0140F43F0020003801400008014097
:1067A0007047704700BFFEE7014802490860704724
:1067B0000030000808ED00E070B504460D46FFF714
:1067C0000FF8A168401AA84206D9A1882068FEF7F0
:1067D000FDFFFFF705F8A06070BD00000EB51C4876
:1067E0001C49086081151B4881600121C16000219E
:1067F00041614FF46021C1610020164948600221C7
:1068000014480161FDF712FD18B1452112A001F0F5
:1068100097FB00200090012001900720029069461C
:106820000C48FDF74FFC18B14F210BA001F088FB7D
:10683000012000900220019007200290694605483F
:10684000FDF740FC18B1592103A001F079FB0EBD02
:1068500000240140EC0000202E2E2F5372632F6184
:1068600064632E630000000010B5124812490860EE
:10687000124800687D2801D1302000E018200E4920
:10688000486000210C488160C1604FF440310161D3
:106890000021416181610121C161002101624162E8
:1068A0008162C162FEF730F818B16A2104A001F0DC
:1068B00047FB10BD00640040B02F0020A80000205E
:1068C0002E2E2F5372632F63616E2E630000000023
:1068D00008B500BF0648406940F00100044948611E
:1068E0000846406900F00100009000BF00BF08BDED
:1068F0000010024000B585B000BF3B48806940F001
:106900002000394988610846806900F02000009025
:1069100000BF00BF00BF0846806940F004008861E6
:106920000846806900F00400009000BF00BF00BF6F
:106930000846806940F0080088610846806900F0D8
:106940000800009000BF00BF002220212748FEF76A
:1069500041FF002280212548FEF73CFF002243F240
:1069600001012348FEF736FFA0200190012002908C
:106970000220049001A91D48FEF79AFD43F2010090
:106980000190012002900220049001A91848FEF70E
:106990008FFD50200190012002900220049001A957
:1069A0001248FEF785FD1348007802280DD16420B7
:1069B000FEF7FCFB012210210C48FEF70BFF012221
:1069C00040210A48FEF706FF0CE06420FEF7EEFBCC
:1069D000002210210548FEF7FDFE00224021034859
:1069E000FEF7F8FE05B000BD0010024000080140AF
:1069F000000C01409C00002010B5084808490860C0
:106A00000320486040F6C41105488160FEF7EEFEA1
:106A100018B13A2103A001F093FA10BD00300040F4
:106A2000E00000202E2E2F5372632F697764672EAB
:106A30006300000010B504460348FFF7E0FC204661
:106A400000F004F810BD00003440002010B50446EA
:106A50000A480B4908600846446000218160C16013
:106A600001610C21416100218161C161FFF786FD57
:106A700018B15C2103A001F063FA10BD0038014099
:106A8000344000202E2E2F5372632F757361727461
:106A90002E63000010B50C480C4908604FF4E1303B
:106AA0004860002109488160C16001610C21416199
:106AB00000218161C161FFF761FD18B14A2104A085
:106AC00001F03EFA10BD000000480040F43F0020F5
:106AD0002E2E2F5372632F75736172742E63000014
:106AE00000BFFEE77047000002480068C0F30220C4
:106AF000704700000CED00E010B5002807DA0A0727
:106B0000140E054A00F00F031B1FD45403E00A07BC
:106B1000130E024A135410BD18ED00E000E400E02B
:106B20007047000010B50446207801280FD1FEF709
:106B300057FE11490968401AB0F57A7F1AD300222E
:106B400001210E48FEF746FE0020207012E020785A
:106B500002280FD1FEF744FE07490968401A40F6A3
:106B6000B831884206D3002201210448FEF732FEE4
:106B70000020207010BD000088000020000C0140A3
:106B800008B508490968C9084FF47A72B1FBF2F1F7
:106B90004143009100BF00BF00994A1E00920029A6
:106BA000F9D108BD000000203EB535480568002435
:106BB00006E0E00025FA00F032490855601CC4B236
:106BC000042CF6DB2E48001D0568002408E0E000D8
:106BD00025FA00F0C1B2201D2A4A1154601CC4B22B
:106BE000042CF4DB264808300568002409E0E000A6
:106BF00025FA00F0C1B204F10800224A1154601CC9
:106C0000C4B2042CF3DB20480568002406E0E00051
:106C100025FA00F01D490855601CC4B2042CF6DBAF
:106C20001948001D0568002408E0E00025FA00F07E
:106C3000C1B2201D154A1154601CC4B2042CF4DBEF
:106C4000114808300568002409E0E00025FA00F04A
:106C5000C1B204F108000D4A1154601CC4B2042CE6
:106C6000F3DB6A460A490748FCF7EAFE0C220749AB
:106C70006846FCF78BFA08B900203EBD0120FCE70E
:106C8000E8F7FF1FB445002000F40008C0450020CD
:106C9000F889000808B5FDF76FF8FEF755FB00BF4F
:106CA00034200B49C86000BF0A48FDF759F80A2094
:106CB000FEF77CFAFEF7E6FA0748009001226946E3
:106CC0000648FDF771F81420FEF770FA08BD0000C1
:106CD0000020024090460020674523010428000858
:106CE00070472DE9F047ADF5007D81468846164690
:106CF0001F46DDF820A24FF4807140A8FCF73BFA54
:106D00004FF480716846FCF736FA0025FCB2552036
:106D10008DF80001AA208DF80101300A8DF80201DA
:106D2000F0B28DF803018DF80481A01CC0B28DF87B
:106D30000501380A8DF806018DF8074122465146B3
:106D400042A8FCF7FFF904F1080240A96846FCF7E5
:106D5000F9F904F108016846FCF756FE0546280ECD
:106D600004F1080140AA5054C5F3074104F1090099
:106D70001154C5F30721401C1154401C1554F02137
:106D8000401C1154401CC2B240A9484600F006FC09
:106D90000DF5007DBDE8F08710B5FEF757FDFFF754
:106DA0002AFB10BD10B594B009200A904FF4803032
:106DB0000B9000200C9001200E901090022011905A
:106DC000C10312914FF4E01113910AA8FFF7C4F820
:106DD00018B1D2211AA001F0B3F80F2005900220BB
:106DE0000690002007904FF48060089000200990E2
:106DF000022105A8FEF76EFF18B1E02110A001F0F6
:106E00009FF8022001908003039001A8FEF7CAFEBC
:106E100018B1E7210AA001F093F8FFF72DF84FF41D
:106E20007A71B0FBF1F42046FFF7CBFA0420FFF7AC
:106E3000B3FA00221146501EFEF7AFFD14B010BD8C
:106E40002E2E2F5372632F6D61696E2E630000002A
:106E50001148006840F001000F490860084640688A
:106E60000E4908400C494860084600680C49084033
:106E7000094908600846006820F480200860084638
:106E8000406820F4FE0048604FF41F008860C8038B
:106E90000449086070470000001002400000FFF83D
:106EA000FFFFF6FE08ED00E010B514480078022858
:106EB0000ED1FEF795FC12490968401A32281BD9F9
:106EC00001200E4908700F480068FFF7B3FD13E07A
:106ED0000A48007801280FD1FEF782FC08490968AA
:106EE000401A41F28831884206D9002003490870CF
:106EF00005480068FFF79EFD10BD00008C000020D3
:106F000090000020A0000020A40000207047000096
:106F100070B588B006460D461446B5F5004F72D0E0
:106F200023DCB5F58A4F6FD00FDCB5F5885F38D01C
:106F30006FF40850284498B3B0F5417F76D0A0F59F
:106F40000450FF38002872D168E0A5F5AA40143833
:106F500000286DD0A0F58050EC38002869D0A0F54D
:106F6000885002380028EED1CAE0B5F5044F75D03C
:106F70000BDCA5F50040A0F5827000286FD0FC283E
:106F80006ED0B0F5007FDED124E1A5F505400438D0
:106F900000287DD0FC287CD0B0F5007FD3D19DE1C6
:106FA0000AE000204FF4885340F2FF720C21009059
:106FB000D948FFF796FEACE1D8480078D0B9FEF783
:106FC0000FFCD74908602078F02808D10120D34968
:106FD000087001221146D348FEF7FCFB0AE0207836
:106FE000F12807D10220CD49087001221146CD4871
:106FF000FEF7F0FB2078F02807D100228021CA4854
:10700000FEF7E8FB09E08DE014E02078F12804D1D8
:1070100001228021C448FEF7DDFB7AE1FFF73AFE4A
:10702000012000F09EFFFEF70BFD72E108E06FE12A
:1070300017E042E0012000F094FFFEF701FD68E157
:1070400005222146B9A0FCF7A1F830B9FEF7C8FB2C
:10705000B84908600220B84908705AE1D4E080E0DD
:1070600090E0B6482168016061684160A168816074
:10707000B348E168016021694160B24A0146AF4806
:10708000FCF7DEFCB048AF490A6802604A6801E0DC
:10709000E2E0FBE04260896881600F22ABA10C3026
:1070A000FCF750F8A84845F21B5340F2FF720C2140
:1070B00000909948FFF715FE2BE1FCF729FDA74842
:1070C000016802914168039180680490A4480168B6
:1070D0000591416806918068079002A846F21863FE
:1070E00040F2FF720C2100908B48FFF7FAFDC82098
:1070F000FEF75CF8012000F034FFFEF7A1FC08E188
:1071000023462A460121974800F066FA3220FEF70E
:107110004DF822462946934800F098FA3220FEF7AF
:1071200045F8F6E001219048FCF704FE8F4908700D
:1071300000208DF81C008DF81D008DF81E000846FB
:1071400000788DF81F0007A848F2040340F2FF7290
:107150000C2100907048FFF7C4FD3220FEF726F89E
:10716000D7E0E078814908707F48FCF7E1FE80A015
:1071700048F2020340F2FF720C2100906648FFF7CC
:10718000B0FDC6E001217848001DFCF7D3FD794928
:10719000086008460068000E8DF81C00084600686C
:1071A000000C8DF81D0008460088000A8DF81E00AE
:1071B000084600788DF81F0007A848F2042340F223
:1071C000FF720C2100905448FFF78BFD3220FDF731
:1071D000EDFF9EE020780006617800EB0140A17889
:1071E00000EB0120E1780844624908605E48FCF742
:1071F0009FFE5FA048F2020340F2FF720C21009054
:107200004548FFF76EFD84E0012157480830FCF740
:1072100091FD5949086008460068000E8DF81C0071
:1072200008460068000C8DF81D0008460088000A1A
:107230008DF81E00084600788DF81F0007A848F258
:10724000044340F2FF720C2100903348FFF749FDE0
:107250003220FDF7ABFF5CE020780006617800EBA0
:107260000140A17800EB0120E17808444249086020
:107270003D48FCF75DFE3EA048F2020340F2FF727B
:107280000C2100902448FFF72CFD42E001213648F4
:107290000C30FCF74FFD3949086008460068000EC5
:1072A0008DF81C0008460068000C8DF81D0008468B
:1072B0000088000A8DF81E00084600788DF81F002F
:1072C00007A848F2046340F2FF720C2100901248B4
:1072D000FFF707FD3220FDF769FF1AE0207800066E
:1072E000617800EB0140A17800EB0120E1780844CF
:1072F000224908601C48FCF71BFE1DA048F202034F
:1073000040F2FF720C2100900348FFF7EAFC00E016
:1073100000BF00BF08B070BD4800002084000020FE
:1073200088000020000C01400008014052455345F0
:1073300054000000900000208C00002072420020C9
:10734000AD0000207E4200208A42002056342E31BB
:107350002E325F323032343039303400B4450020C0
:10736000C045002070000020002C00089C00002078
:107370004F4B0000A0000020A4000020A800002027
:1073800070B505466C6A0020E085E0842046FFF772
:107390004DF870BD10B50A46C38893421EDB0369E1
:1073A0001B68DB6823F0200304692468E360C3885A
:1073B0009B1AC38003691B68DB6843F020030469E0
:1073C0002468E360114683880B4499B203888B429A
:1073D00002DC0388CB1A99B281801CE003691B6828
:1073E000DB6823F0200304692468E360C18800237C
:1073F000C38003691B68DB6843F0200304692468C9
:10740000E36083880B4499B203888B4202DC0388D3
:10741000CB1A99B2818010BD0168C96821F49071BE
:107420000268D1600168496921F001010268516177
:10743000202180F83A10704710B504462068C068D3
:1074400020F040002168C860202084F839002046E0
:10745000FFF7A7F9002010BD00BFC28803889A4239
:10746000FBD002691268D26822F0800203691B68AF
:10747000DA60C2888AB9026912681268C2F3C0125F
:107480005AB102691268516002691268D26842F00A
:10749000800203691B68DA6070474388C268D15470
:1074A0004288521C92B2428003889A4201D1002243
:1074B0004280C288521CC28002691268D26842F0BF
:1074C000800203691B68DA6000BFE5E710B5024679
:1074D0000B461946D4889C4209DB94880C44A1B21F
:1074E00014888C4204DC14880C1BA1B200E000213B
:1074F000D468605C10BD70B5044694F83A00222848
:107500004AD1A068B0F5805F13D1A56A206940B95F
:1075100020684068C0F308002880A06A801CA06230
:1075200019E020684068C0B22880A06A401CA062B0
:1075300011E0206938B920684068C1B2A26A501CC5
:10754000A062117007E02068406800F07F01A26A25
:10755000501CA0621170E08D401E80B2E085C8B959
:107560002068C06820F020002168C8602068C068DA
:1075700020F480702168C8602068406920F0010014
:1075800021684861202084F83A002046FFF708F976
:10759000002070BD0020FCE70220FAE7F0B50546A8
:1075A0000E461746286900680949884204D10948EF
:1075B0000078012800D1F0BD002405E0315D2846A7
:1075C000FFF74AFF601CC4B2BC42F7DB00BFF2E722
:1075D000003801409C0000202DE9F047C0B08246F1
:1075E0000F46164698464FF480716846FBF7C3FD78
:1075F00000240025A14614258DF800708DF8015057
:10760000300A8DF8020000BF06E018F80410E01CF4
:107610000DF80010601CC4B2F0B2A042F5DC0024EA
:1076200005E01DF8040080EA0909601CC4B2AC4200
:10763000F7DB09F0FF01681E0DF800102A466946C5
:107640005046FFF7ABFF40B0BDE8F0872DE9F043AF
:10765000C1B081460F4690464FF4807101A8FBF7F8
:107660008AFD0024002500260D2555208DF80400F4
:1076700000BF05E018F80410601C01AA1154C4B240
:10768000F8B2A042F6DC002409E001A9601C085C05
:10769000095D00EB012080B24640A01CC4B20A2C58
:1076A000F3DBE81E01AA16543112A81E1154F02172
:1076B000681E11542A4601A94846FFF76FFF41B0E2
:1076C000BDE8F0832DE9F0410446002520680069FB
:1076D00020F44050E1680843216808612169A068EE
:1076E00008436169084305432068C06841F20C61A2
:1076F000884328432168C8602068406920F44070AE
:10770000A1690843216848615F49206888425CD1CB
:10771000FEF7C8FB00EBC00101EB001061688900B7
:10772000B0FBF1F6FEF7BEFB00EBC00101EB001071
:1077300061688900B0FBF1F06421B0FBF1F000EB6F
:10774000C00101EB0010A6EB8000322101EB00101C
:107750006421B0FBF1F000F0F006FEF7A3FB00EBB4
:10776000C00101EB001061688900B0FBF1F06421F9
:10777000B0FBF1F006EB0016FEF794FB00EBC00146
:1077800001EB001061688900B0FBF1F7FEF78AFB9E
:1077900000EBC00101EB001061688900B0FBF1F063
:1077A0006421B0FBF1F000EBC00101EB0010A7EB8E
:1077B0008000322101EB00106421B0FBF1F000F0F9
:1077C0000F003044216888605BE0FEF75BFB00EB54
:1077D000C00101EB001061688900B0FBF1F6FEF713
:1077E00051FB00EBC00101EB001061688900B0FBA8
:1077F000F1F06421B0FBF1F000EBC00101EB0010EF
:10780000A6EB8000322101EB00106421B0FBF1F007
:1078100000F0F006FEF736FB00EBC00101EB0010B4
:1078200061688900B0FBF1F06421B0FBF1F006EB78
:107830000016FEF727FB00EBC00101EB00106168AA
:107840008900B0FBF1F7FEF71DFB00EBC00101EB77
:10785000001061688900B0FBF1F06421B0FBF1F029
:1078600000EBC00101EB0010A7EB8000322101EB1F
:1078700000106421B0FBF1F000F00F0030442168EB
:107880008860BDE8F0810000003801402DE9FF4F1D
:10789000C1B0894692461E46DDF83CB14E9F4FF47A
:1078A000807101A8FBF767FC00250024A046381D65
:1078B000C4B2F72C00DDF7243A208DF804008DF8CF
:1078C00005908DF806A08DF80740300A8DF8080065
:1078D000F0B28DF80900380A8DF80A00F8B28DF878
:1078E0000B00002507E01BF8051005F1080001AAB0
:1078F0001154681CC5B2201FA842F4DC012506E023
:1079000001A8405D40441FFA80F8681CC5B2201DE4
:107910008542F5DB01AA02F800804FEA2821601DAC
:1079200011540D21A01D11540A21E01D1154401CB9
:10793000C2B201A94198FFF731FE45B0BDE8F08F12
:10794000014691F8390021282CD18868B0F5805F74
:107950000FD10A6A1088C0F308000B6858600869E4
:1079600018B9086A801C086209E0086A401C0862AD
:1079700005E00B6A581C086218780B685860C88CC0
:10798000401E80B2C88458B90868C06820F08000E2
:107990000B68D8600868C06840F040000B68D86089
:1079A000002070470220FCE710B5054800F020F8E1
:1079B000044800F052F80448FEF73AFD10BD0000FC
:1079C0005C000020700000203440002010B5054805
:1079D00000F00EF8044800F040F80448FEF728FDD7
:1079E00010BD00003400002048000020F43F0020BB
:1079F00008B5026912681268C2F3401262B30269E4
:107A000012685268D1B20269126812680022B2B9D3
:107A10004388C268D1544288521C92B24280038883
:107A20009A4201DB00224280C288521C92B2C2807C
:107A300003889A4203DD0288C2800122027200BFDD
:107A400000220092026912681268009202691268AC
:107A50005268009200BF00BF08BD0169096809684B
:107A6000C1F3C01139B301690968C96801F0800127
:107A700009B36FF08001026912681160C18891B189
:107A8000C188491EC1808288C168895C0269126808
:107A900051608188491C89B28180028891420ADB49
:107AA0000021818007E001690968C96821F080012F
:107AB00002691268D160704710B50248FCF7FAFD00
:107AC00010BD0000B02F00202DE9F34F87B0804695
:107AD000002005900490B8F8060008287EDB0021FD
:107AE0004046FFF7F3FC8246BAF13A0F77D1012105
:107AF0004046FFF7EBFC8146B9F1FA0F70D1022145
:107B00004046FFF7E3FC0746112F03D0162F01D0A4
:107B10000C2F66D103214046FFF7D8FC0446B8F885
:107B2000061004F1080081421DDA6048007801283F
:107B300006D1FDF755FE5E49086000205B490870DC
:107B4000FDF74EFE5A490968411A0898814207D943
:107B500098F806104046FFF71DFC012053490870B5
:107B600009B0BDE8F08FFDF73BFE524908600120E7
:107B70004E490870002607E0F1B24046FFF7A6FC28
:107B80004D498855701C86B2201D8642F4DBC1B277
:107B90004046FFF79BFC8346601DC1B24046FFF79D
:107BA00095FC0BEB002080B20490012607E04248D0
:107BB000815D0598084480B20590701C86B2201D36
:107BC0008642F4DBA01DC1B24046FFF77FFC039064
:107BD000E01DC1B24046FFF779FC03E064E05FE0DE
:107BE00059E053E00290DDE90401884249D103984D
:107BF0000D2846D102980A2843D12F4A121D294642
:107C00003846FFF783F9042C17DB2B4840792A49C3
:107C1000097900EB012080B206902748C0792649F7
:107C2000897900EB012085B2234808302B4600906B
:107C300039462248069AFFF754F84CF2091085425B
:107C40000FD04CF2022085420BD04CF2023085421C
:107C500007D04CF20240854203D04CF202508542DC
:107C600003D1FDF7BDFD1649086004F10800C1B25B
:107C70004046FFF78FFB4FF400511248FDF7A6FD79
:107C800012E001214046FFF785FB0DE0012140464F
:107C9000FFF780FB08E001214046FFF77BFB03E094
:107CA00001214046FFF776FB00BF59E7BC000020EA
:107CB000B800002098000020A542002048000020C5
:107CC00090000020000C01402DE9F34F87B0814661
:107CD000B9F806000D287BDB00214846FFF7F6FBCC
:107CE000039090490398087001214846FFF7EEFB86
:107CF00082468C4981F801A00398552869D1BAF1D0
:107D0000AA0FFBD102214846FFF7E0FB85498870A6
:107D100003214846FFF7DAFB8249C8700846C0785D
:107D2000897800EB012080B2069004214846FFF7D5
:107D3000CDFB05467B490D71112D03D0162D01D0C9
:107D40000C2D7DD105214846FFF7C0FB074675483D
:107D5000477107214846FFF7B9FB8346062148468D
:107D6000FFF7B4FB0BEB00201FFA80F84FEA182056
:107D70006C49887181F8078007214846FFF7A6FB08
:107D80000446381B02287DD1B9F8061007F10B0014
:107D900081421FDA64480078012806D1FDF720FDF2
:107DA00062490860002060490870FDF719FD5F49CD
:107DB0000968411A0898814207D999F8061048467F
:107DC000FFF7E8FA01205849087009B0BDE8F08FC4
:107DD000A5E0A0E001205449087000260FE006F15C
:107DE0000800C1B24846FFF771FB51498855084663
:107DF000815D06F108004B4A1154701C86B2A64200
:107E0000EDDB04F10800C1B24846FFF75FFB4FEA23
:107E1000006B04F10900C1B24846FFF757FB0BEBBA
:107E2000004B04F10A00C1B24846FFF74FFB0BEBD1
:107E3000002B04F10B00C1B24846FFF747FB00E0FE
:107E400064E00BEB0001049104F108013548FBF7F5
:107E5000DBFD0590DDE90410081A4DD1344A414696
:107E60002846FFF755F8221D2E49091D881EFBF7ED
:107E700069F904F10800C1B24846FFF727FBA11DCC
:107E8000284A00E03DE05054C81CC1B24846FFF704
:107E90001DFBE11D234A5054C81CC1B24846FFF7E0
:107EA00015FB04F108011F4A5054C81CC1B24846D2
:107EB000FFF70CFB04F109011A4A5054F02104F1B8
:107EC0000A001154421C17490698FBF7E3FC1848B6
:107ED000CDE900802A46FA211648069BFFF7D6FC1A
:107EE00007F10B00C1B24846FFF754FA4FF40051B6
:107EF0001148FDF76BFC68E701214846FFF74AFA95
:107F00000DE001214846FFF745FA08E00121484607
:107F1000FFF740FA03E001214846FFF73BFA00BFB4
:107F200053E70000A3440020C4000020C00000204C
:107F3000A443002070000020000C014000BFFEE7B9
:107F400000BFFEE702E008C8121F08C1002AFAD1EC
:107F500070477047002001E001C1121F002AFBD1C9
:107F6000704700F0010181F31388704710B50A468D
:107F7000038993421EDB1E4B1B685B6923F00203DF
:107F80001B4C2468636103899B1A0381184B1B688F
:107F90005B6943F00203164C246863611146C38891
:107FA0000B4499B243888B4202DC4388CB1A99B2C6
:107FB000C1801CE00E4B1B685B6923F002030C4C74
:107FC00024686361018900230381094B1B685B6995
:107FD00043F00203064C24686361C3880B4499B2E2
:107FE00043888B4202DC4388CB1A99B2C18010BD12
:107FF000B02F002010B502460B46194614899C424A
:1080000009DBD4880C44A1B254888C4204DC548827
:108010000C1BA1B200E00021D468605C10BD000020
:108020007FB50646002404E0305D18490855601C01
:10803000C4B2082CF8DB3823154A02A9304600F0F8
:1080400091F900241EE0002504E002A800F04AF99E
:10805000681CC5B20F48005DA842F6DC40230E4AFA
:10806000694602A800F07EF9002507E06846405DF9
:10807000E1000A4A89184855681CC5B2082DF5DB8D
:10808000601CC4B2102CDEDB7FBD0000D5000020D8
:10809000C08A0008988D0008F88A00080046002071
:1080A000FFB587B00F4600250AE0785D3349495D8A
:1080B000884203D03846FFF7B3FF0725681CC5B2D6
:1080C000082DF2DB40232E4A05A9079800F04AF953
:1080D000012538E0002405E005A8005D03A9085546
:1080E000601CC4B2082CF7DB0998002805D1681E73
:1080F000C00024494018009005E01020401BC0003B
:10810000204940180090002406E003A9201D085CC7
:1081100005A90855601CC4B2042CF6DB01AA05A908
:10812000009800F033F8002409E003A8005D01A9DD
:10813000095D484005AA211D5054601CC4B2042C9E
:10814000F3DB681CC5B2112DC4DB6846067D017ED9
:1081500001750676467D417E41754676867D817E37
:1081600081758676C67DC17EC175C6764023064A76
:1081700005A80A9900F0F6F80BB0F0BDD500002074
:10818000008A000800460020408A0008F0B587B049
:1081900005460E4617464023114A05A9304600F011
:1081A000E1F8002411E005A8005D295D4840800643
:1081B000800E03A90855A0010A49401803A9095DCA
:1081C000405C01A90855601CC4B2082CEBDB2023DD
:1081D000054A394601A800F0C5F807B0F0BD000017
:1081E000388B0008988B0008788B0008FEF7DCFAC3
:1081F000FDF738FBFEF7D6FDFBF708FDFEF77AFB2F
:10820000FEF766FBFEF7EAFAFEF72EFBFEF7F4FB3D
:1082100029480068FEF71AFCFEF73CFCFBF7C0F9A2
:10822000FBF780F8C820FCF7C1FF24484088B0F570
:108230007A7F04DA012220212148FDF7CBFAFEF7EC
:10824000B3FC2049087035E01F48FDF7F7FA4FF4FA
:10825000FA611E48FFF738FC4FF4FA611C48FFF73B
:1082600033FD1C48FEF75EFC16480078C0B90024B8
:1082700000BF09E004EB4401174A02EBC100C8212A
:10828000FBF7D0F9601C84B2162CF3DBFA211348FB
:10829000FEF792FA4FF47A711148FEF78DFA07E073
:1082A00064210E48FEF788FA64210D48FEF784FA2F
:1082B000FEF7FAFDC8E70000A4000020040000203B
:1082C00000080140C5000020E00000205C00002004
:1082D0003400002084000020A02D00200800002091
:1082E000180000200CB5002104E0425C6B465A5493
:1082F0004A1CD1B20829F8DB002112E0425C520688
:10830000120E425406290ADA6B464A1C9A5C8023F4
:108310001A40802A03D1425C01231A4342544A1C6A
:10832000D1B20729EADB6A46127880231A40002A74
:1083300004D0C27810231A43C27003E0C27810231D
:108340009A43C2706A46D27808231A40002A04D0A1
:10835000827901231A43827103E082795208520024
:1083600082710CBDFFB5124C002000BF00260546EF
:10837000401C4E550828F9DB002000BF1378521C22
:10838000DE10009DAD5D5E07760FA65D3540002DC9
:1083900007D0C5104D5D4607760FA65D3543C61064
:1083A0008D55451C2846039EB542E7DBFFBD000006
:1083B000A88D000800000000000000000102030476
:1083C0000607080900000000010203041007120755
:1083D000130714071507150620072107230724078D
:1083E00025073007310732073407350735064007C0
:1083F0004107420743074507000021104220633030
:108400008440A550C660E770088129914AA16BB1EC
:108410008CC1ADD1CEE1EFF1311210027332522294
:10842000B5529442F772D662399318837BB35AA33C
:10843000BDD39CC3FFF3DEE3622443342004011464
:10844000E664C774A44485546AA54BB5288509958C
:10845000EEE5CFF5ACC58DD5533672261116300634
:10846000D776F6669556B4465BB77AA719973887DC
:10847000DFF7FEE79DD7BCC7C448E5588668A778F4
:108480004008611802282338CCC9EDD98EE9AFF92C
:10849000488969990AA92BB9F55AD44AB77A966AD4
:1084A000711A500A333A122AFDDBDCCBBFFB9EEB7C
:1084B000799B588B3BBB1AABA66C877CE44CC55CA4
:1084C000222C033C600C411CAEED8FFDECCDCDDDCC
:1084D0002AAD0BBD688D499D977EB66ED55EF44E74
:1084E000133E322E511E700E9FFFBEEFDDDFFCCF1C
:1084F0001BBF3AAF599F788F8891A981CAB1EBA170
:108500000CD12DC14EF16FE18010A100C230E320EB
:108510000450254046706760B9839893FBA3DAB393
:108520003DC31CD37FE35EF3B1029012F322D2323B
:108530003542145277625672EAB5CBA5A895898563
:108540006EF54FE52CD50DC5E234C324A01481048B
:108550006674476424540544DBA7FAB79987B89733
:108560005FE77EF71DC73CD7D326F2369106B016DB
:1085700057667676154634564CD96DC90EF92FE9F3
:10858000C899E9898AB9ABA944586548067827682B
:10859000C018E1088238A3287DCB5CDB3FEB1EFBD3
:1085A000F98BD89BBBAB9ABB754A545A376A167A7B
:1085B000F10AD01AB32A923A2EFD0FED6CDD4DCDA3
:1085C000AABD8BADE89DC98D267C076C645C454CCB
:1085D000A23C832CE01CC10C1FEF3EFF5DCF7CDF73
:1085E0009BAFBABFD98FF89F176E367E554E745E1B
:1085F000932EB23ED10EF01E00000000B71DC10444
:108600006E3B8209D926430DDC7604136B6BC517CC
:10861000B24D861A0550471EB8ED08260FF0C92244
:10862000D6D68A2F61CB4B2B649B0C35D386CD31AC
:108630000AA08E3CBDBD4F3870DB114CC7C6D04878
:108640001EE09345A9FD5241ACAD155F1BB0D45B54
:10865000C2969756758B5652C836196A7F2BD86EBC
:10866000A60D9B6311105A6714401D79A35DDC7D34
:108670007A7B9F70CD665E74E0B6239857ABE29C20
:108680008E8DA191399060953CC0278B8BDDE68F54
:1086900052FBA582E5E66486585B2BBEEF46EABA3C
:1086A0003660A9B7817D68B3842D2FAD3330EEA934
:1086B000EA16ADA45D0B6CA0906D32D42770F3D098
:1086C000FE56B0DD494B71D94C1B36C7FB06F7C3CC
:1086D0002220B4CE953D75CA28803AF29F9DFBF6C4
:1086E00046BBB8FBF1A679FFF4F63EE143EBFFE5AC
:1086F0009ACDBCE82DD07DEC77708634C06D4730C4
:10870000194B043DAE56C539AB0682271C1B4323CB
:10871000C53D002E7220C12ACF9D8E1278804F1643
:10872000A1A60C1B16BBCD1F13EB8A01A4F64B05AB
:108730007DD00808CACDC90C07AB9778B0B6567C77
:1087400069901571DE8DD475DBDD936B6CC0526F53
:10875000B5E6116202FBD066BF469F5E085B5E5ABB
:10876000D17D1D576660DC5363309B4DD42D5A4933
:108770000D0B1944BA16D84097C6A5AC20DB64A8E7
:10878000F9FD27A54EE0E6A14BB0A1BFFCAD60BB53
:10879000258B23B69296E2B22F2BAD8A98366C8E3B
:1087A00041102F83F60DEE87F35DA9994440689D33
:1087B0009D662B902A7BEA94E71DB4E0500075E497
:1087C000892636E93E3BF7ED3B6BB0F38C7671F7CB
:1087D000555032FAE24DF3FE5FF0BCC6E8ED7DC2C3
:1087E00031CB3ECF86D6FFCB8386B8D5349B79D1AB
:1087F000EDBD3ADC5AA0FBD8EEE00C6959FDCD6D19
:1088000080DB8E6037C64F643296087A858BC97ECE
:108810005CAD8A73EBB04B77560D044FE110C54B3E
:10882000383686468F2B47428A7B005C3D66C158AE
:10883000E4408255535D43519E3B1D252926DC2192
:10884000F0009F2C471D5E28424D1936F550D83256
:108850002C769B3F9B6B5A3B26D6150391CBD407B6
:1088600048ED970AFFF0560EFAA011104DBDD01436
:10887000949B93192386521D0E562FF1B94BEEF59A
:10888000606DADF8D7706CFCD2202BE2653DEAE656
:10889000BC1BA9EB0B0668EFB6BB27D701A6E6D336
:1088A000D880A5DE6F9D64DA6ACD23C4DDD0E2C036
:1088B00004F6A1CDB3EB60C97E8D3EBDC990FFB972
:1088C00010B6BCB4A7AB7DB0A2FB3AAE15E6FBAACE
:1088D000CCC0B8A77BDD79A3C660369B717DF79FBE
:1088E000A85BB4921F4675961A163288AD0BF38CAE
:1088F000742DB081C330718599908A5D2E8D4B594E
:10890000F7AB085440B6C95045E68E4EF2FB4F4ACD
:108910002BDD0C479CC0CD43217D827B9660437F3D
:108920004F460072F85BC176FD0B86684A16476CAD
:1089300093300461242DC565E94B9B115E565A1591
:1089400087701918306DD81C353D9F0282205E0655
:108950005B061D0BEC1BDC0F51A69337E6BB5233B5
:108960003F9D113E8880D03A8DD097243ACD562035
:10897000E3EB152D54F6D4297926A9C5CE3B68C161
:10898000171D2BCCA000EAC8A550ADD6124D6CD255
:10899000CB6B2FDF7C76EEDBC1CBA1E376D660E735
:1089A000AFF023EA18EDE2EE1DBDA5F0AAA064F435
:1089B000738627F9C49BE6FD09FDB889BEE0798D71
:1089C00067C63A80D0DBFB84D58BBC9A62967D9ECD
:1089D000BBB03E930CADFF97B110B0AF060D71ABBD
:1089E000DF2B32A66836F3A26D66B4BCDA7B75B8AD
:1089F000035D36B5B440F7B121402324255E262A15
:108A000039312921191109013B332B231B130B0386
:108A10003D352D251D150D053F372F271F170F0736
:108A200038302820181008003A322A221A120A0276
:108A30003C342C241C140C043E362E261E160E0626
:108A400027072F0F37173F1F26062E0E36163E1EFE
:108A500025052D0D35153D1D24042C0C34143C1C0E
:108A600023032B0B33133B1B22022A0A32123A1A1E
:108A7000210129093111391920002808301038182E
:108A80002122232425262728292A2B2C2D2E2F305E
:108A90003132333435363738393A3B3C3D3E3F404E
:108AA0000102030405060708090A0B0C0D0E0F103E
:108AB0001112131415161718191A1B1C1D1E1F202E
:108AC00038302820181008003931292119110901DE
:108AD0003A322A221A120A023B332B233E362E2622
:108AE0001E160E063D352D251D150D053C342C2476
:108AF0001C140C041B130B0300000D04100A1700B8
:108B0000000002091B0E051400001607120B0319C2
:108B100000000F01061A130C00002836331E242E05
:108B200000001D2F27322C2000002B343026372147
:108B300000002D1F2931231C00001F040001020327
:108B400000000308040506070000070C08090A0BCB
:108B500000000B100C0D0E0F00000F14101112135B
:108B600000001318141516170000171C18191A1BEB
:108B700000001B001C1D1E1F1F0E272C3C17372436
:108B8000041E2E350C253E15050F2F1D3F360614ED
:108B9000261C3D0D2D1607340E040D01020F0B0887
:108BA000030A060C05090007000F07040E020D0159
:108BB0000A060C0B0905030804010E080D06020B3A
:108BC0000F0C0907030A05000F0C0802040901072E
:108BD000050B030E0A00060D0F01080E060B030419
:108BE0000907020D0C00050A030D04070F02080E09
:108BF0000C00010A06090B05000E070B0A040D0103
:108C000005080C060903020F0D080A01030F0402F0
:108C10000B06070C00050E090A00090E06030F05D6
:108C2000010D0C070B0402080D0700090304060AD6
:108C30000208050E0C0B0F010D060409080F0300B6
:108C40000B01020C050A0E07010A0D0006090807B0
:108C5000040F0E030B05020C070D0E030006090A94
:108C6000010208050B0C040F0D080B05060F00038D
:108C70000407020C010A0E090A0609000C0B070D75
:108C80000F01030E05020804030F00060A010D0878
:108C90000904050B0C07020E020C0401070A0B065F
:108CA0000805030F0D000E090E0B020C04070D0141
:108CB00005000F0A030908060402010B0A0D070844
:108CC0000F090C050603000E0B080C07010E020D20
:108CD000060F00090A0405030C010A0F0902060821
:108CE000000D03040E07050B0A0F0402070C09050B
:108CF00006010D0E000B0308090E0F0502080C03F8
:108D00000700040A010D0B060403020C09050F0AF3
:108D10000B0E01070600080D040B020E0F00080DD4
:108D2000030C0907050A06010D000B070409010AD7
:108D30000E03050C020F080601040B0D0C03070EB1
:108D40000A0F060800050902060B0D0801040A07B0
:108D50000905000F0E02030C0D020804060F0B019B
:108D60000A09030E05000C07010F0D080A0307048A
:108D70000C05060B000E0902070B0401090C0E027C
:108D800000060A0D0F03050802010E07040A080D6C
:108D90000F0C09000305060B010102020202020288
:108DA00001020202020202018040201008040201B6
:108DB000D08D000800000020E0000000447F000883
:108DC000B08E0008E0000020C0490000547F000879
:108DD00000A24A0400000000000C01400010000046
:108DE0000000000000000000000C01400020000016
:108DF0000000000000000000010000000000000072
:108E0000010000000004000000000000000000005D
:108E1000F42F0020F43F00200004000000000000B8
:108E200000000000F4330020F43F002000040000A4
:108E30000000000000000000F43700203440002053
:108E4000000400000000000000000000F43B0020CF
:108E5000344000200000000000000000000000007E
:108E60000000000000000000000000000100000001
:108E700000E1000080250000FA0000000000000072
:108E800000000000000000000000000001000000E1
:108E9000000000000101000000F0FFFF00000000E2
:108EA00010000000010000000000000000000000B1
:04000005080030EDD2
:00000001FF
